:020000040000FA
:0600000088EF1EF0120063
:0A0006000100783D0000FA00000040
:0400100006000000E6
:0C0014000001806B8051006E016A200E1C
:10002000005C000E015815E28051EA6A600FE96E2B
:10003000000EEA22EF50E66E8051E66EE66A9FEC13
:100040001DF0E552E552E552B6EC1EF00001802BA2
:10005000E3D71200000EE66EE66AFFEC1DF0E552F3
:10006000E5520001606F0F0E605D36E00F0E606FAD
:10007000616B626B010E636F6469656966696769CC
:10008000686B020E696F6A6B6B6F6C6B6D6F940EB1
:100090006E6F020E6F6F940E706F020E716F940E82
:1000A000726F020E736F880E746F130E756F880E69
:1000B000766F130E776F880E786F130E796FD00EF0
:1000C0007A6F070E7B6FD00E7C6F070E7D6F050E6B
:1000D0007E6F7F6F9FDF1ED0010E816F8151006E9A
:1000E000016A200E005C000E015814E28151E66E98
:1000F000E66AFFEC1DF0E552E552E66E0001815123
:10010000EA6A600FE96E000EEA22E552E750EF6EF0
:10011000812BE4D71200090EE66E040EE66EED0E9A
:10012000E66E0EEC1DF0E552E552E55292809282A9
:10013000928492869288928A1200D9CFE6FFE1CF0C
:10014000D9FFFE0EDBCFE6FF4BEC1EF0E5520C0EA6
:10015000E66E96EC1EF0E552B9EC1EF0B1EC1EF026
:10016000000901E0FBD7A1EC1EF000D0E552E7CF7B
:10017000D9FF12004D0EE66EE66A2C0EE66EC9EC53
:100180001CF0E552E552E5521200D9CFE6FFE1CF6F
:10019000D9FFFE0EDBCFE6FF34EC1EF0E552ACA239
:1001A000FED7E552E7CFD9FF1200D9CFE6FFE1CF66
:1001B000D9FFFD0EDBCF00F0FE0EDBCF01F0070E06
:1001C000D89001320032E804FBE17F0E0014E66EA5
:1001D000DCDFE5527F0EE76EFD0EDBCF00F0FE0E9A
:1001E000DBCF01F0E7500016016A0050E66ECDDF6C
:1001F000E552E552E7CFD9FF1200D9CFE6FFE1CFB4
:10020000D9FFFD0EDBCF00F0DB06FE0EDBCF01F0E9
:1002100001E2DB060050011006E00C0EE66E78EC01
:100220001EF0E552EED7E552E7CFD9FF1200870E58
:10023000E66E83DFE552F3CF85F0F4CF86F08F0EC4
:10024000E66E7BDFE552F3CF87F0F4CF88F0970EB0
:10025000E66E73DFE552F3CF89F0F4CF8AF09F0E9C
:10026000E66E6BDFE552F3CF8BF0F4CF8CF0A70E88
:10027000E66E63DFE552F3CF8DF0F4CF8EF0AF0E74
:10028000E66E5BDFE552F3CF8FF0F4CF90F0120013
:10029000D9CFE6FFE1CFD9FFFE0EDB50EA6A620F4D
:1002A000E96E000EEA22EFCF00F0060E005C1AE2C3
:1002B000FE0EDB50EA6A620FE96E000EEA22EF34AE
:1002C000EA6AFE0BEA36E96E850EE926000EEA229E
:1002D000EECF00F0EFCF01F000C0F3FF01C0F4FF5C
:1002E0000CD00BD0FC0EDBCF00F0FD0EDBCF01F00D
:1002F00000C0F3FF01C0F4FF00D0E552E7CFD9FF03
:1003000012000001010E9F6F826BAA6B030EAA5DA3
:100310000EE2AA51E96EEA6AD890E936EA36910E01
:10032000E926000EEA22EE68ED68AA2BEFD7170E39
:10033000E66EE3EC1DF0E5521200D9CFE6FFE1CF07
:10034000D9FFFE0EEA6ADB34FE0BEA36E96E9B0E3D
:10035000E926000EEA22EECF00F0EFCF01F0FF0E0B
:10036000001802E1FF0E011801E1BDD0FE0EEA6A9D
:10037000DB34FE0BEA36E96E910EE926000EEA2226
:10038000FF0EEE1802E1FF0EED1801E0ACD0FE0EFC
:10039000EA6ADB34FE0BEA36E96EFA0EE926000E55
:1003A000EA22EE50ED101CE1FE0EEA6ADB34FE0B91
:1003B000EA36E96E9B0EE926000EEA22EECF00F047
:1003C000EFCF01F0FE0EEA6ADB34FE0BEA36E96E8F
:1003D000AB0EE926000EEA2200C0EEFF01C0EDFFE1
:1003E000FE0EEA6ADB34FE0BEA36E96EAB0EE92656
:1003F000000EEA22EECF00F0EFCF01F0FE0EEA6A27
:10040000DB34FE0BEA36E96E9B0EE926000EEA228B
:100410000001EE50005CB16FEE500158B26FD88011
:10042000B25104E7FE0EB15DFF0EB25915E3B235CD
:1004300004E2B1510208000EB2550EE3FE0EEA6A64
:10044000DB34FE0BEA36E96EFA0EE926000EEA22EC
:10045000EE2A000EEF220CD0FE0EEA6ADB34FE0B11
:10046000EA36E96EFA0EE926000EEA22EE6AED6A35
:10047000FE0EEA6ADB34FE0BEA36E96EFA0EE92676
:10048000000EEA22EECF00F0EFCF01F01E0E005C6E
:10049000000E015828E3FE0EEA6ADB34FE0BEA3652
:1004A000E96EAB0EE926000EEA22EECF00F0EFCFA8
:1004B00001F0FE0EEA6ADB34FE0BEA36E96E910EBD
:1004C000E926000EEA2200C0EEFF01C0EDFFFE0E9D
:1004D000EA6ADB34FE0BEA36E96EFA0EE926000E14
:1004E000EA22EE6AED6AE552E7CFD9FF1200828474
:1004F0009EDEC4EC1DF0F3CFC8F0F4CFC9F00001CC
:100500009F5103E0836B846B6FD0CA51C85D836FCA
:10051000CB51C959846F400E1E6E1F6A83C023F0F1
:1005200084C024F0DFEC13F01CC0C4F01DC0C5F083
:10053000030E236E246AC4C01EF0C5C01FF062EC17
:100540001EF01EC0C4F01FC0C5F00001C66BC76B13
:10055000C735000EC71909E6D880FF0EC455FF0E37
:10056000C555000EC655000EC75505E2046805685E
:10057000066A076A08D0C4C004F0C5C005F0C6C04A
:1005800006F0C7C007F0D8900750000A08E6000E32
:10059000045C000E0558000E0658000E075805E2D0
:1005A000006A016A026A036A1BD0C735000EC719C8
:1005B00009E6D880FF0EC455FF0EC555000EC6557E
:1005C000000EC75505E200680168026A036A08D098
:1005D000C4C000F0C5C001F0C6C002F0C7C003F03F
:1005E00000C083F001C084F0C8C0CAF0C9C0CBF01D
:1005F000822B68C0E6FF69C0E6FFE66A49DEE55285
:10060000E552E552F3CF97F0F4CF98F06AC0E6FFD9
:100610006BC0E6FF010EE66E3BDEE552E552E552A9
:10062000F3CF99F0F4CF9AF0E668E668030EE66E31
:100630002FDEE552E552E552F3CF9BF0F4CF9CF06C
:10064000E668E668040EE66E23DEE552E552E55202
:10065000F3CF9DF0F4CF9EF00001B36BB3510108CE
:1006600002E28DEF08F0B351E96EEA6AD890E936FC
:10067000EA36970EE926000EEA22EECF0EF0EFCF13
:100680000FF0B351E96EEA6AD890E936EA36680E9F
:10069000E926000EEA22EE500E5C0C6EEE500F586A
:1006A0000D6E0CC01EF00DC01FF075EC12F01DC0D9
:1006B00008F01EC009F01FC00AF020C00BF0226A2B
:1006C000400E236E9C0E246E450E256E08C01DF054
:1006D00009C01EF00AC01FF00BC020F072EC13F02E
:1006E0001DC004F01EC005F01FC006F020C007F0BA
:1006F000226AC00E236E7F0E246E440E256E04C047
:100700001DF005C01EF006C01FF007C020F01FEC52
:1007100013F01DC000F01EC001F01FC002F020C089
:1007200003F00001B351E96EEA6AD890E936EA367F
:100730006E0EE926000EEA22EECF14F0EFCF15F090
:1007400014C01EF015C01FF073EC12F01DC010F0A5
:100750001EC011F01FC012F020C013F010C022F014
:1007600011C023F012C024F013C025F000C01DF00A
:1007700001C01EF002C01FF003C020F01FEC13F0F8
:100780001DC0B8F01EC0B9F01FC0BAF020C0BBF049
:10079000010EB3C0E7FFE75204E0E846FE0BE706B0
:1007A000FCE10001611518E0226A236A800E246EC4
:1007B000BF0E256EB8C01DF0B9C01EF0BAC01FF044
:1007C000BBC020F072EC13F01DC0B8F01EC0B9F031
:1007D0001FC0BAF020C0BBF0006A016A800E026E32
:1007E000BF0E036E086A096A800E0A6E3F0E0B6E1A
:1007F000B8C022F0B9C023F0BAC024F0BBC025F0C5
:1008000008C01DF009C01EF00AC01FF00BC020F088
:1008100035EC14F0010A07E1046A056A800E066EE1
:100820003F0E076E08D0B8C004F0B9C005F0BAC0DA
:1008300006F0BBC007F004C022F005C023F006C0DC
:1008400024F007C025F000C01DF001C01EF002C05A
:100850001FF003C020F02CEC14F0010A08E10001A5
:10086000C06BC16B800EC26FBF0EC36F2AD00C6A03
:100870000D6A800E0E6E3F0E0F6EB8C022F0B9C02A
:1008800023F0BAC024F0BBC025F00CC01DF00DC091
:100890001EF00EC01FF00FC020F035EC14F0010A5E
:1008A00008E10001C06BC16B800EC26F3F0EC36FC9
:1008B00008D0B8C0C0F0B9C0C1F0BAC0C2F0BBC067
:1008C000C3F0006A016A7A0E026E440E036E00C025
:1008D000E6FF01C0E6FF02C0E6FF03C0E6FFC0C0BE
:1008E000E6FFC1C0E6FFC2C0E6FFC3C0E6FF78EC8A
:1008F0001DF0E552E552E552E552E552E7CF03F02F
:10090000E552E7CF02F0E552E7CF01F0E552E7CF3D
:1009100000F01CC004F01DC005F01EC006F01FC092
:1009200007F004C022F005C023F006C024F007C081
:1009300025F000C01DF001C01EF002C01FF003C072
:1009400020F072EC13F01DC0BCF01EC0BDF01FC043
:10095000BEF020C0BFF0B3C0E6FFEFDCE5520001FF
:10096000B351E96EEA6AD890E936EA36910EE92683
:10097000000EEA22EECF00F0EFCF01F0FF0E0018DC
:1009800002E1FF0E011801E1BAD0B351E96EEA6A43
:10099000D890E936EA369B0EE926000EEA22EECF21
:1009A00002F0EFCF03F0FF0E021802E1FF0E031872
:1009B00001E1A5D0B351E96EEA6AD890E936EA368A
:1009C0009B0EE926000EEA22EECF0AF0EFCF0BF0E5
:1009D000B351E96EEA6AD890E936EA36910EE92613
:1009E000000EEA22EE500A5C086EEE500B58096EBB
:1009F00008C01EF009C01FF075EC12F01DC004F015
:100A00001EC005F01FC006F020C007F03B0E226E8E
:100A10009C0E236EA60E246E470E256E04C01DF09C
:100A200005C01EF006C01FF007C020F072EC13F0E6
:100A30001DC000F01EC001F01FC002F020C003F076
:100A4000030E0001B325E96EEA6AD890E936EA366A
:100A50006E0EE926000EEA22EECF10F0EFCF11F075
:100A600010C01EF011C01FF073EC12F01DC00CF08E
:100A70001EC00DF01FC00EF020C00FF00CC022F001
:100A80000DC023F00EC024F00FC025F000C01DF0F3
:100A900001C01EF002C01FF003C020F01FEC13F0D5
:100AA0001DC0B4F01EC0B5F01FC0B6F020C0B7F036
:100AB000030E0001B325006E010E005204E0E8466B
:100AC000FE0B0006FCE10001611518E0226A236AB2
:100AD000800E246EBF0E256EB4C01DF0B5C01EF092
:100AE000B6C01FF0B7C020F072EC13F01DC0B4F018
:100AF0001EC0B5F01FC0B6F020C0B7F004D0B46B74
:100B0000B56BB66BB76B00019F5113E0B351040D89
:100B1000F3CFE9FFF4CFEAFFA20EE926000EEA22A6
:100B2000BCC0EEFFBDC0EEFFBEC0EEFFBFC0EEFF1B
:100B300042D183C01EF084C01FF073EC12F01DC0C0
:100B400000F01EC001F01FC002F020C003F0226AB6
:100B5000240E236E740E246E490E256E00C01DF007
:100B600001C01EF002C01FF003C020F01FEC13F004
:100B70001DC0C0F01EC0C1F01FC0C2F020C0C3F035
:100B8000C0C022F0C1C023F0C2C024F0C3C025F011
:100B9000B4C01DF0B5C01EF0B6C01FF0B7C020F045
:100BA00072EC13F01DC0C0F01EC0C1F01FC0C2F037
:100BB00020C0C3F00001B351EA6A7E0FE96E000E57
:100BC000EA22EFCF04F004C01FF062EC12F01DC067
:100BD00000F01EC001F01FC002F020C003F00001B1
:100BE000B351040DF3CFE9FFF4CFEAFFA20EE926DB
:100BF000000EEA22EECF09F0EECF0AF0EECF0BF0B6
:100C0000EFCF0CF0C0C022F0C1C023F0C2C024F06E
:100C1000C3C025F009C01DF00AC01EF00BC01FF0B4
:100C20000CC020F089EC12F01DC005F01EC006F0CB
:100C30001FC007F020C008F005C022F006C023F056
:100C400007C024F008C025F000C01DF001C01EF050
:100C500002C01FF003C020F072EC13F01DC0C0F002
:100C60001EC0C1F01FC0C2F020C0C3F0BCC022F043
:100C7000BDC023F0BEC024F0BFC025F0C0C01DF031
:100C8000C1C01EF0C2C01FF0C3C020F089EC12F03A
:100C90001DC0C0F01EC0C1F01FC0C2F020C0C3F014
:100CA0000001B351EA6A7E0FE96E000EEA22EF28D6
:100CB000046E04C01FF062EC12F01DC000F01EC0F4
:100CC00001F01FC002F020C003F000C022F001C0FC
:100CD00023F002C024F003C025F0C0C01DF0C1C045
:100CE0001EF0C2C01FF0C3C020F01FEC13F01DC0E7
:100CF000C0F01EC0C1F01FC0C2F020C0C3F0226A05
:100D0000236A246A256AC0C01DF0C1C01EF0C2C09B
:100D10001FF0C3C020F035EC14F0010A16E0226A7F
:100D2000236A246A3F0E256EC0C01DF0C1C01EF0AC
:100D3000C2C01FF0C3C020F089EC12F0FDEC13F02C
:100D40001EC004F01FC005F015D0226A236A246A71
:100D50003F0E256EC0C01DF0C1C01EF0C2C01FF006
:100D6000C3C020F088EC12F0FDEC13F01EC004F0BC
:100D70001FC005F004C01EF005C01FF075EC12F096
:100D80001DC000F01EC001F01FC002F020C003F023
:100D90000001B351040DF3CFE9FFF4CFEAFFA20E37
:100DA000E926000EEA2200C0EEFF01C0EEFF02C0FD
:100DB000EEFF03C0EEFFB351040DF3CFE9FFF4CF14
:100DC000EAFFA20EE926000EEA22EECF00F0EECFF7
:100DD00001F0EECF02F0EFCF03F0D40E226EE20E60
:100DE000236EA60E246E3D0E256E00C01DF001C0C0
:100DF0001EF002C01FF003C020F072EC13F01DC003
:100E0000C0F01EC0C1F01FC0C2F020C0C3F0006A15
:100E1000016AFE0E026E420E036E0001B351E96ECE
:100E2000EA6AD890E936EA367A0EE926000EEA2216
:100E3000EECF10F0EFCF11F010C01EF011C01FF078
:100E400073EC12F01DC00CF01EC00DF01FC00EF0B0
:100E500020C00FF00CC022F00DC023F00EC024F013
:100E60000FC025F0C0C01DF0C1C01EF0C2C01FF0F1
:100E7000C3C020F072EC13F01DC008F01EC009F0D2
:100E80001FC00AF020C00BF0226A236A7A0E246E7B
:100E9000440E256E08C01DF009C01EF00AC01FF0E8
:100EA0000BC020F01FEC13F01DC004F01EC005F0B5
:100EB0001FC006F020C007F004C022F005C023F0D8
:100EC00006C024F007C025F000C01DF001C01EF0D0
:100ED00002C01FF003C020F089EC12F01DC0C0F06A
:100EE0001EC0C1F01FC0C2F020C0C3F0226A236A36
:100EF000246A256AC0C01DF0C1C01EF0C2C01FF028
:100F0000C3C020F035EC14F0010A16E0226A236A0F
:100F1000246A3F0E256EC0C01DF0C1C01EF0C2C0C5
:100F20001FF0C3C020F089EC12F0FDEC13F01EC0DE
:100F300004F01FC005F015D0226A236A246A3F0E10
:100F4000256EC0C01DF0C1C01EF0C2C01FF0C3C0DE
:100F500020F088EC12F0FDEC13F01EC004F01FC06E
:100F600005F0053404E20450FF08000E055403E2C6
:100F70000268036A3BD0226A236A246A256AC0C0D9
:100F80001DF0C1C01EF0C2C01FF0C3C020F035EC80
:100F900014F0010A16E0226A236A246A3F0E256EC5
:100FA000C0C01DF0C1C01EF0C2C01FF0C3C020F001
:100FB00089EC12F0FDEC13F01EC002F01FC003F02C
:100FC00015D0226A236A246A3F0E256EC0C01DF028
:100FD000C1C01EF0C2C01FF0C3C020F088EC12F0E8
:100FE000FDEC13F01EC002F01FC003F0D8900350B8
:100FF00004E6000E025C000E035803E2006A016A78
:1010000080D0226A236A246A256AC0C01DF0C1C04C
:101010001EF0C2C01FF0C3C020F035EC14F0010A6E
:1010200016E0226A236A246A3F0E256EC0C01DF0B6
:10103000C1C01EF0C2C01FF0C3C020F089EC12F086
:10104000FDEC13F01EC006F01FC007F015D0226A99
:10105000236A246A3F0E256EC0C01DF0C1C01EF079
:10106000C2C01FF0C3C020F088EC12F0FDEC13F0FA
:101070001EC006F01FC007F0073404E20650FF0848
:10108000000E075403E20068016A3BD0226A236A1B
:10109000246A256AC0C01DF0C1C01EF0C2C01FF086
:1010A000C3C020F035EC14F0010A16E0226A236A6E
:1010B000246A3F0E256EC0C01DF0C1C01EF0C2C024
:1010C0001FF0C3C020F089EC12F0FDEC13F01EC03D
:1010D00000F01FC001F015D0226A236A246A3F0E77
:1010E000256EC0C01DF0C1C01EF0C2C01FF0C3C03D
:1010F00020F088EC12F0FDEC13F01EC000F01FC0D1
:1011000001F00001B351EA6AA00FE96E000EEA2275
:1011100000C0EFFFB32B2EEF03F09F6B8294120001
:1011200094949368F19E8A68BAEC00F02AEC00F07F
:101130008BEC00F081EC01F00001CC6BCD6BCE6B41
:10114000CF6BF46B17EC0AF06DEC0AF002D8FCD709
:101150001200200E0101005D03E36D50020B01E05F
:10116000E9D00001CC51CD1102E1000E08D0CCC075
:10117000E9FFCDC0EAFFEF50800B01E0010E00094E
:1011800001E089D077EC02F00001F76BA0C0D0F04D
:10119000A1C0D1F0811CD26FF4C0D3F0F4511DE195
:1011A000F66BF651006E016A150E005C000E0158D8
:1011B00014E2F651EA6A820FE96E000EEA22EF505D
:1011C000E66E040EF625EA6AD00FE96E000EEA22FA
:1011D000E552E750EF6EF62BE4D7F4051DE1F66B10
:1011E000F651006E016A200E005C000E015814E2F8
:1011F000F651EA6A600FE96E000EEA22EF50E66EE1
:10120000040EF625EA6AD00FE96E000EEA22E552D6
:10121000E750EF6EF62BE4D7F66B240EF65D26E270
:10122000F651EA6AD00FE96E000EEA22EFCF00F025
:10123000F651EA6A510FE96E040EEA22EF50005CA3
:1012400013E0F651EA6AD00FE96E000EEA22EF5081
:10125000E66EF651EA6A510FE96E040EEA22E55293
:10126000E750EF6E010EF76FF62BD7D7F75113E06B
:10127000240EE66E510EE66E040EE66E010EE66E6C
:10128000E66ECDEC11F0006E050EE15E0050F3CF7E
:10129000CCF0F4CFCDF00001CE51CF1102E1000E21
:1012A00008D0CEC0E9FFCFC0EAFFEF50800B01E0CD
:1012B000010E00093EE10401305102E131C4F4F0B5
:1012C000300524E10001F66BF651006E016A200E34
:1012D000005C000E015813E2F629EA6A300FE96E4D
:1012E000040EEA22EF50E66EF651EA6A600FE96EEC
:1012F000000EEA22E552E750EF6EF62BE5D70AEC36
:1013000000F02AEC00F00001010EF46F210EE66EF1
:10131000300EE66E040EE66EE66A010EE66ECDEC69
:1013200011F0006E050EE15E0050F3CFCEF0F4CF69
:10133000CFF000D0120012001200120012009CEF39
:101340001BF012001E0EE66E010EE66E27EC11F089
:10135000E552E552210EE66E300EE66E040EE66EA4
:10136000E66A010EE66ECDEC11F0006E050EE15E50
:101370000050F3CFCEF0F4CFCFF012006D84000117
:10138000080EF86F070EF96FF807000EF95BF851B9
:10139000F911FAE16D941200D9CFE6FFE1CFD9FF40
:1013A000FD0EDBCF1EF0FE0EDBCF1FF0010E1E1870
:1013B00001E11F5033E0E8681E1802E1E8681F18D9
:1013C0002BE0030E1E1801E11F5024E0040E1E182E
:1013D00001E11F501DE0020E1E1801E11F5016E032
:1013E000170E1E1801E11F500FE0160E1E1801E126
:1013F0001F5008E0150E1E1801E11F5001E010D02B
:10140000A1DF0FD09EDF0DD09ADF0BD096DF09D081
:1014100092DF07D091DF05D091DF03D0000001D02B
:0E14200000D0010E00D0E552E7CFD9FF120038
:02142E00D9CF14
:10143000E6FFE1CFD9FFE6526A6A686A9F0E6B6EDB
:10144000FB0E696E6D8C6D9C6E6A000EE66EE66A30
:10145000E66A710EE66E0F0EE66E1AEC1EF0006E76
:10146000050EE15E0050DF6ADF50006E016A080E73
:10147000005C000E015810E2DF50040DF3CFE9FFCD
:10148000F4CFEAFF000EE926040EEA22EE6AEE6AC5
:10149000EE6AEE6ADF2AE8D7160E706E68A60CD0E8
:1014A000030EE66E680EE66E0F0EE66E46EC12F068
:1014B000E552E552E552F2D70101136B186B196B37
:1014C0001A6B6D98080E0B6F040E0C6F016B006B9E
:1014D000E552E552E7CFD9FF1200D9CFE6FFE1CFC1
:1014E000D9FFE652A19A0101005111E105D06D6AC0
:1014F000696A0101006BC9D06D6A696A6DB602D074
:101500006D86FCD70101010E006F160E6F6E00058F
:1015100008E16DBA06D0686A696A69806988020E56
:10152000006F6850040B0FE06950040B0CE0020ED2
:10153000E66E680EE66E0F0EE66E46EC12F0E552B1
:10154000E552E552E6D86DB2A0D06850010B1BE021
:101550006950010B18E06BDF0101040E006F0401FC
:10156000200E026F040E036F080E016F006B8C0ECD
:101570000013E66A680EE66E0F0EE66E46EC12F099
:10158000E552E552E5526850100B0FE06950100B20
:101590000CE0A3D8040EE66E680EE66E0F0EE66E43
:1015A00046EC12F0E552E552E5526850400B1DE062
:1015B0006950400B1AE0010EE66EE66A000EE66E18
:1015C000E66A020EE66EE66ACCEC09F0006E060EE4
:1015D000E15E0050060EE66E680EE66E0F0EE66ED9
:1015E00046EC12F0E552E552E5526850200B04E05B
:1015F0006950200B01E04ED86850020B12E0695090
:10160000020B0FE0010EE66EE66A000EE66EE66A79
:10161000E668E668CCEC09F0006E060EE15E00506C
:101620006A6A040E0101005D01E22FD069A62DD087
:10163000DF6A040EDF5C29E268A624D06CCF20F1BB
:10164000030EE66E680EE66E0F0EE66E46EC12F0C6
:10165000E552E552E552780E0101201502E178D8F5
:1016600010D0000EE66EE66A200EE66E010EE66E03
:10167000010EE66EE66ACCEC09F0006E060EE15E45
:10168000005001D002D0DF2AD4D7E552E552E7CF8F
:10169000D9FF120070A015D003C1E9FF04C1EAFF11
:1016A000EF5080080DE10BC1E9FF0CC1EAFFEF50DC
:1016B000840806E103C1E9FF04C1EAFF8C0EEF6E66
:1016C0007090050EE66E680EE66E0F0EE66E46EC46
:1016D00012F0E552E552E55212006984040EE66EFE
:1016E000680EE66E0F0EE66E46EC12F0E552E5521D
:1016F000E5526D82000EE66EE66AE66EE66A040E5C
:10170000E66EE66ACCEC09F0006E060EE15E005073
:1017100012006D92000EE66EE66AE66EE66A030E51
:10172000E66EE66ACCEC09F0006E060EE15E005053
:10173000699468A40CD0020EE66E680EE66E0F0E79
:10174000E66E46EC12F0E552E552E552F2D7120091
:10175000FD0E0101201520E17E0E2015E8407F0BD3
:10176000040DF3CF03F1F4CF04F1000E0327040EB0
:10177000042303C105F104C106F1057503C1E9FFA6
:1017800004C1EAFFEF503C0BE842E8420D0802E1D9
:1017900009D801D02AD805D0FD0E2015040801E192
:1017A0002DD812000BC1E9FF0CC1EAFFEF50800BEE
:1017B00005E00BC1E9FF0CC1EAFFEF6A01010F6B05
:1017C000106B146B156B136B04D9000EE66EE66A92
:1017D000E66EE66A170EE66EE66ACCEC09F0006E7D
:1017E000060EE15E005096EF0EF0020E0101105D54
:1017F00003E1F3EC0FF001D04ED81200D9CFE6FF91
:10180000E1CFD9FFE6520BC1E9FF0CC1EAFFEF506F
:10181000400B01E0010EDF6E01010B75080E005D4B
:101820000AE122C46EFF6E50000803E2100E006F42
:1018300002D0040E006F100528E10BC1E9FF0CC1B6
:10184000EAFF020EE926000EEA22280EEE6E040ED2
:10185000ED6E3EDB020E01010F5D07E10BC1E9FFFA
:101860000CC1EAFF840EEF6E0FD0DF5007E10BC111
:10187000E9FF0CC1EAFFC80EEF6E06D00BC1E9FF0D
:101880000CC1EAFF880EEF6E01D005D8E552E55293
:10189000E7CFD9FF1200D9CFE6FFE1CFD9FF030E82
:1018A000E126020E0101105D4AE16D50100B47E088
:1018B00003C1E9FF04C1EAFFEE52EF50006E016A76
:1018C000080E001801E101503AE103C1E9FF04C12B
:1018D000EAFFEF503C0BE842E8420D0830E105C159
:1018E000E9FF06C1EAFFEF50800B29E105C1E9FFDE
:1018F00006C1EAFF020EE926000EEA22200EEE6E75
:10190000040EED6EDF6ADF50006E016A080E005CA7
:10191000000E015813E2DF50EA6A280FE96E040E48
:10192000EA22EF50E66EDF50EA6A200FE96E040EFD
:10193000EA22E552E750EF6EDF2AE5D731D0106B8F
:1019400005C1E9FF06C1EAFFEE52080EEF6E05C1C0
:10195000E9FF06C1EAFF020EE926000EEA22200E88
:10196000EE6E040EED6E05C1E9FF06C1EAFF8C0EB6
:10197000EF6E0BC1E9FF0CC1EAFFEF6A040E0B1911
:10198000006E0CC101F0010E00C0DBFF020E01C0B1
:10199000DBFF010EDBCFE9FF020EDBCFEAFFEF6AD0
:1019A000010118AF0CD01B511C1107E005D01CC160
:1019B000FAFF01011B51F96EFADF0101189F030EB6
:1019C000E15C02E2E16AE552E16EE552E7CFD9FF60
:1019D000120004012051600BE842E842E842E8426C
:1019E000E842000901E058D021510C0A54E00B0AEA
:1019F00043E00C0A35E0010A26E00B0A22E0020A65
:101A000020E0030A1CE0080A10E0010A0CE00F0ABB
:101A100008E0030A01E03FD00101138F080E006FB8
:101A20003BD0C8D839D070DB37D00101010E116F1F
:101A3000010E126F1381010E146F138F2DD014D964
:101A40002BD02BD829D024510101116F126B020E1B
:101A50001127010E12231381010E146F138F1CD056
:101A60000101138F04012451EA6A020FE96E010E8D
:101A7000EA2222C4EFFF10D0000EE66EE66AE66EA0
:101A8000E66A160EE66EE66ACCEC09F0006E060E0B
:101A9000E15E005001D000D01200D9CFE6FFE1CFC7
:101AA000D9FF040EE1260401220510E120511F0B8D
:101AB00000090CE10101138F030E0401215D04E113
:101AC0000101010E1F6F02D001011F6B04012251A1
:101AD00067E120511F0B020863E124510F0B00093D
:101AE0005FE00101138F040124BF10D024510F0BBC
:101AF000E96EEA6AD890E936EA36070EE926010E61
:101B0000EA22EECFDEFFEDCFDDFF0FD024510F0B29
:101B1000E96EEA6AD890E936EA360B0EE926010E3C
:101B2000EA22EECFDEFFEDCFDDFF030E215D07E100
:101B3000DECFE9FFDDCFEAFF840EEF6E31D0245116
:101B40000F0B016A700F006E0F0E0122020E00C013
:101B5000DBFF030E01C0DBFF020EDBCFE9FF030E4C
:101B6000DBCFEAFFEE90ED5224AF0DD0DECFE9FFE0
:101B7000DDCFEAFFEF6ADF74DECFE9FFDDCFEAFFFA
:101B8000400EEF6E0DD0DECFE9FFDDCFEAFF880E0D
:101B9000EF6EDF74DECFE9FFDDCFEAFFC80EEF6E38
:101BA000040EE15C02E2E16AE552E16EE552E7CF44
:101BB000D9FF1200800E0401205D55E10101C00E25
:101BC000136F04012351030A2EE0010A0EE0030AF9
:101BD00003E00101136B47D00101240E116F380E91
:101BE000126F120E146F156B3ED02251F66EF76A0B
:101BF000D890F636F736EB0EF626380EF7220900A7
:101C0000F5CF11F10A00F5CF12F1020E0101F76ACA
:101C10001125F66E1251F7220900F5CF14F10A00D2
:101C2000F5CF15F120D0030E225D1AE22251F66E97
:101C3000F76AD890F636F736ED0EF626380EF7220C
:101C40000900F5CF11F10A00F5CF12F111C1F6FF2D
:101C500012C1F7FF0800F5500101146F156B02D097
:101C60000101136B00D01200D9CFE6FFE1CFD9FFFD
:101C7000020EE1260401286B296B20511F0B020A7A
:101C800013E0030A0EE0010A01E03CD00101138FCA
:101C900002D00401288101011F0502E1040128830B
:101CA00031D00101138F2ED00101138F040124BF05
:101CB00010D024510F0BE96EEA6AD890E936EA3663
:101CC000070EE926010EEA22EECFDEFFEDCFDDFFA3
:101CD0000FD024510F0BE96EEA6AD890E936EA3644
:101CE0000B0EE926010EEA22EECFDEFFEDCFDDFF7F
:101CF000DECFE9FFDDCFEAFFEF50040B02E0010E7B
:101D0000286F00D0010113AF07D0280E116F040E09
:101D1000126F1381020E146F020EE15C02E2E16A9F
:101D2000E552E16EE552E7CFD9FF12006D9801014F
:101D300013BF4AD018AF28D0020E106F0BC1E9FFB5
:101D40000CC1EAFFEE52EF6A0BC1E9FF0CC1EAFFDA
:101D5000C80EEF6E05C1E9FF06C1EAFFEE52080E9C
:101D6000EF6E05C1E9FF06C1EAFF020EE926000E8B
:101D7000EA22280EEE6E040EED6E05C1E9FF06C1E3
:101D8000EAFFC80EEF6E1FD005C1E9FF06C1EAFFEA
:101D9000EE52080EEF6E05C1E9FF06C1EAFF020E22
:101DA000E926000EEA22200EEE6E040EED6E05C14D
:101DB000E9FF06C1EAFF8C0EEF6E0BC1E9FF0CC113
:101DC000EAFF840EEF6E83D018BF81D0040120AFEC
:101DD00056D0010114510401265D01011551040181
:101DE000275904E226C414F127C415F171D8010162
:101DF000010E106F05C1E9FF06C1EAFFEE52080EA1
:101E0000EF6E05C1E9FF06C1EAFF020EE926000EEA
:101E1000EA22200EEE6E040EED6E05C1E9FF06C14A
:101E2000EAFF800EEF6E03C1E9FF04C1EAFFEE5244
:101E3000080EEF6E03C1E9FF04C1EAFF020EE926B6
:101E4000000EEA22200EEE6E040EED6E03C1E9FFD5
:101E500004C1EAFF800EEF6E0BC1E9FF0CC1EAFF7F
:101E6000020EE926000EEA22280EEE6E040EED6E3A
:101E70000BC1E9FF0CC1EAFFC80EEF6E28D00101CB
:101E8000020E106F0BC1E9FF0CC1EAFFEE52EF6AC0
:101E90000BC1E9FF0CC1EAFFC80EEF6E05C1E9FFF7
:101EA00006C1EAFFEE52080EEF6E05C1E9FF06C15A
:101EB000EAFF020EE926000EEA22280EEE6E040E5C
:101EC000ED6E05C1E9FF06C1EAFFC80EEF6E120014
:101ED000D9CFE6FFE1CFD9FF020EE1260101080EBE
:101EE000145D000E15590EE214C1DEFF15C1DDFFB1
:101EF0000F5103E1010E0F6F04D00F0502E1020E36
:101F00000F6F03D0080EDE6EDD6A0BC1E9FF0CC156
:101F1000EAFFEF920BC1E9FF0CC1EAFFEF900BC1A2
:101F2000E9FF0CC1EAFF010EDB50EF120BC1E9FF24
:101F30000CC1EAFFEE52DFCFEFFF000EDB50145F63
:101F4000010EDB50155B280E1D6F040E1E6F13B1C2
:101F500021D0D9CFE9FFDACFEAFFEE50ED1019E03A
:101F600011C1F6FF12C1F7FF112B000E122308005A
:101F7000F550E66E1DC1E9FF1EC1EAFF1D2B000EE4
:101F80001E23E552E750EF6EDF06010E01E2DB068D
:101F9000E0D71FD0D9CFE9FFDACFEAFFEE50ED103E
:101FA00018E011C1E9FF12C1EAFF112B000E122344
:101FB000EF50E66E1DC1E9FF1EC1EAFF1D2B000EAA
:101FC0001E23E552E750EF6EDF06010E01E2DB064D
:101FD000E1D7020EE15C02E2E16AE552E16EE55210
:101FE000E7CFD9FF1200D9CFE6FFE1CFD9FF020E2C
:101FF000E12603C1E9FF04C1EAFFEE52EFCFDFFFA4
:10200000DFCF00F000500101195D000E1A5903E204
:1020100019C1DFFF09D0DF50006E016A0050195D61
:10202000196F01501A591A6F010EDB6ADF50F36EF7
:10203000010EDBCFF4FFF350F45C16E2010EDB502F
:10204000EA6A280FE96E040EEA22EF50E66E16C126
:10205000E9FF17C1EAFF162B000E1723E552E750E0
:10206000EF6E010EDB2AE2D7000ED8801955000E64
:102070001A5528E205C1E9FF06C1EAFFEE52080E33
:10208000EF6E05C1E9FF06C1EAFF020EE926000E68
:10209000EA22280EEE6E040EED6E03C1E9FF04C1C4
:1020A000EAFFEF50400B07E105C1E9FF06C1EAFF77
:1020B000C80EEF6E06D005C1E9FF06C1EAFF880E23
:1020C000EF6E18D005C1E9FF06C1EAFF020EE9264E
:1020D000000EEA22200EEE6E040EED6E1B511C1156
:1020E00007E005D01CC1FAFF01011B51F96EFADFB0
:1020F0000101189F020EE15C02E2E16AE552E16E25
:10210000E552E7CFD9FF12000101138F000EE66EF2
:10211000E66AE66A710EE66E0F0EE66E1AEC1EF0C7
:10212000006E050EE15E0050010EE66EE66AE66A9C
:10213000020EE66E010EE66E1AEC1EF0006E050E43
:10214000E15E005022C401F10401225104E10101C9
:10215000100E006F11D00101200E006F000EE66E10
:10216000E66AE66EE66A150EE66EE66ACCEC09F003
:10217000006E060EE15E00501200D9CFE6FFE1CFFF
:10218000D9FF020EE126000EDE6E040EDD6EFD0E9E
:10219000DB50E824026EFE0EDB50040DF3500224E7
:1021A000040DF350006E016A020E0F0B05E0D8908B
:1021B00001320032E806FBE1D89000360136D890B3
:1021C00000360136D9CFE9FFDACFEAFF0050EE261C
:1021D0000150ED22DECFE9FFDDCFEAFFEF9EFD0EDD
:1021E000DB500FE1FE0EEA6ADB34FE0BEA36E96EE5
:1021F000070EE926010EEA22DECFEEFFDDCFEDFF6E
:102200000ED0FE0EEA6ADB34FE0BEA36E96E0B0EE8
:10221000E926010EEA22DECFEEFFDDCFEDFFDECFB5
:10222000E9FFDDCFEAFFEF9CDECFE9FFDDCFEAFF7C
:10223000040EE926000EEA22EF8C020EE15C02E2B7
:10224000E16AE552E16EE552E7CFD9FF1200D9CF3E
:10225000E6FFE1CFD9FF020EE126FE0EDB50016A58
:10226000700F006E0F0E012200C0DEFF01C0DDFF07
:10227000DECFE9FFDDCFEAFFFD0EDBCFEFFFDBA412
:1022800007D0E66AFE0EDBCFE6FF77DFE552E552C8
:10229000FD0EDBA208D0010EE66EFE0EDBCFE6FFE0
:1022A0006CDFE552E552020EE15C02E2E16AE552C2
:1022B000E16EE552E7CFD9FF1200D9CFE6FFE1CFBB
:1022C000D9FF020EE126FE0EDB5020E105C1E9FF39
:1022D00006C1EAFFEE52080EEF6E05C1E9FF06C126
:1022E000EAFF020EE926000EEA22200EEE6E040E30
:1022F000ED6E05C1E9FF06C1EAFF8C0EEF6E0BC162
:10230000E9FF0CC1EAFF840EEF6E3DD0FD0EDB50FD
:10231000E824026EFE0EDB50040DF3500224040D7F
:10232000F3CF00F0F4CF01F0000E0026040E0122DE
:1023300000C0DEFF01C0DDFF840E006EDECFE9FFCE
:10234000DDCFEAFF0050EF12FD0EDB50E824026EF5
:10235000FE0EDB50040DF3500224010F040DF3CFE9
:1023600000F0F4CF01F0000E0026040E012200C0A0
:10237000DEFF01C0DDFF840E006EDECFE9FFDDCFA2
:10238000EAFF0050EF12020EE15C02E2E16AE55260
:10239000E16EE552E7CFD9FF1200D9CFE6FFE1CFDA
:1023A000D9FF020EE126FD0EDB500FE0FE0EEA6AB9
:1023B000DB34FE0BEA36E96E0B0EE926010EEA224B
:1023C000EECFDEFFEDCFDDFF0ED0FE0EEA6ADB348E
:1023D000FE0BEA36E96E070EE926010EEA22EECF81
:1023E000DEFFEDCFDDFFDECFE9FFDDCFEAFF020E3E
:1023F000E926000EEA22FB0EDBCFEEFFFC0EDBCF60
:10240000EDFFDECFE9FFDDCFEAFFEE52FA0EDBCFC4
:10241000EFFF400E006EDECFE9FFDDCFEAFF005098
:10242000EF16880E006EDECFE9FFDDCFEAFF005029
:10243000EF12FD0EDB500CE0FE0EEA6ADB34FE0B01
:10244000EA36E96E0B0EE926010EEA22EF740BD094
:10245000FE0EEA6ADB34FE0BEA36E96E070EE92669
:10246000010EEA22EF74DECF00F0DDCF01F000C0F4
:10247000F3FF01C0F4FF020EE15C03E200D0E16A69
:10248000E552E16EE552E7CFD9FF1200D9CFE6FF62
:10249000E1CFD9FF010EF36EFC0EDB5004E0D890C3
:1024A000F336E806FCE1F350E81C006EFD0EDBCFCE
:1024B000E9FFFE0EDBCFEAFF0050EF16E552E7CF53
:0424C000D9FF12002E
:0C24C400179E05D0179E1FAE02D01F6CA3
:1024D000178E1FC019F0186A296A286A860E1A6EAC
:1024E0001B6AAFEF14F0179E08D0179E1FAE05D0E1
:1024F0001E6C1F1EE86A1F22178E1FC019F01EC017
:1025000018F0296A286A8E0E1A6E1B6AAFEF14F053
:10251000257E176AEBEC14F003EC15F017B693EF79
:1025200014F017A20AD017AA03D017BE93EF14F025
:1025300017A49FEF14F09CEF14F017AA05D017AC66
:102540009FEF14F09CEF14F017A00AD017A808D042
:1025500017BE04D017A402D0A8EF14F0ACEF14F00B
:10256000286A1B6A2550205C276E10E31DC029F0E5
:102570001EC018F01FC019F020C026F022C01DF0A8
:1025800023C01EF024C01FF0173A09D022C029F042
:1025900023C018F024C019F025C026F0276C179E20
:1025A00017BC178E26C01AF017B0DBEF14F01A0E06
:1025B0002760DBEF14F01A6A206A17A408D01D6C9C
:1025C0001E1E1F1E201EE86A1E221F22202217AC7C
:1025D00008D0296C181E191E1A1EE86A1822192222
:1025E0001A221C6A275207E020341F321E321D3285
:1025F0001C32272EF9D71D5029261E5018221F5095
:10260000192220501A221CC028F0179E1AAE0BD097
:10261000286C291E181E191E1A1EE86A2922182263
:1026200019221A22178E1AA006D0D8801932183211
:1026300029322832262A26C01AF0AFEF14F0176A82
:10264000EBEC14F003EC15F017B693EF14F017A2AF
:1026500005D017BA93EF14F09AEF14F017BAA6EF5B
:1026600014F017A005D017B893EF14F0A6EF14F0EC
:1026700017B89AEF14F01B6A7F0E20241A6EE86ACE
:102680001B2225501A5EE86A1B5A1A0E266E206A13
:10269000286A296A186A196A22501D5E23501E5A38
:1026A00024501F5A000E205A09E722501D2623509D
:1026B0001E2224501F22000E202201D0288AD890EA
:1026C0001D361E361F362036D89028362936183645
:1026D0001936262EE1D71F501E101D10D8A4288AA7
:1026E000AFEF14F0176AEBEC14F003EC15F017B62B
:1026F00093EF14F017A205D017B893EF14F09AEFE8
:1027000014F017AA05D017B093EF14F09AEF14F055
:1027100017B002D017A802D0A6EF14F01B6A2550FC
:1027200020241A6EE86A1B227E0E1A5EE86A1B5A83
:10273000286A296A186A196A24501F02F4CF19F00E
:10274000F3CF18F023501F02F3502926F45018221B
:10275000000E192224501E02F3502926F45018228C
:10276000000E192222501F02F3502826F45029226D
:10277000000E1822192223501E02F3502826F4506E
:102780002922000E1822192224501D02F350282657
:10279000F4502922000E1822192222501E02F45051
:1027A0002826000E29221822192223501D02F45037
:1027B0002826000E292218221922AFEF14F01EC07D
:1027C00028F01E502302F4CF1DF0F3CF1CF01F5051
:1027D0002402F4CF1FF0F3CF1EF02302F3501D2686
:1027E000F4501E22E86A1F2228502402F3501D26AE
:1027F000F4501E22E86A1F22000C176AEBEC14F05A
:1028000017B607EF14F017A20ED017B405D07F0E3D
:102810001F6EFF0E1E6E1FD0800E1F6E1E6A1BD015
:102820001F6A1E6A18D017B0FBD78F0E2060EDD735
:102830007E0E2064F5D78E0E205C05E0D8901F3206
:102840001E32202AF8D717A406D01E6C1F1EE86A75
:102850001F221FAEE5D712003EEC14F017B6000C95
:1028600017B0000C17B4000C010C3EEC14F017B6B6
:10287000000C17B0000C17A4000C010C176AEBEC4D
:1028800014F003EC15F017B6120017AE08D017A01D
:1028900004D017A802D017801200179012002550FC
:1028A000205C0BE124501F5C08E123501E5C05E115
:1028B00022501D5C02E117801200D8A002D0178EB2
:1028C00010D0205025C020F0256E1F5024C01FF0CE
:1028D000246E1E5023C01EF0236E1D5022C01DF01A
:1028E000226E2550205C10E0FF0F09E0179017B40E
:1028F00003D017AE1784120017AE17941200252AC2
:10290000D89024322332223222501D5E23501E5A88
:1029100024501F5A1FBEEAD7D8901D361E361F36C8
:10292000202EF8D7C8D77F0E206EFF0E1F6E1E6EAA
:102930001D6E12007F0E17BEFF0E206E02D07F0E9E
:10294000206E800E1F6E1E6A1D6AF3D717AE04D06C
:10295000800E206E1F6AF7D7206A1F6AF4D71950BD
:10296000181029102810F8E01BBEF0D719BE0CD0A3
:102970001A501B10EBE0D890283629361836193635
:102980001A06D8A01B06F2D71B50D4E11A28D2E0B1
:1029900028AE11D07F0E281402E129A00CD0292ADC
:1029A000E86A1822192207E3D8801932183229322E
:1029B0001A2A1A28BFE01A50C9E029C01DF018C011
:1029C0001EF019341F6E1A30206E1F32209E17BE63
:1029D000208E99EF14F01F36203602E31784177EFD
:1029E00006E11780206A1F6A1E6A1D6A12002028ED
:1029F00003E0D8801F321200D8901F3202E1178204
:102A00001200178612002436253602E3178C177E33
:102A100006E11788256A246A236A226A120025289B
:102A200003E0D88024321200D8902432EAE1178AD9
:102A30001200166A24AE22EF15F0236C241EE86AF9
:102A40002422161E1FAE2AEF15F01E6C1F1EE86A08
:102A50001F22161E62EC1EF01FBE3AEF15F016AED6
:102A6000000C1E6C1F1EE86A1F221A6C1B1EE86AEF
:0E2A70001B22000C16BE31EF15F01788FF0C6C
:022A7E00D9CFAE
:102A8000E6FFDACFE6FFE1CFD9FFE2CFDAFF210E92
:102A9000E12402E3E168E652E16ED950FA0FE96EF3
:102AA000FF0E04DAD950050FE66E000EDA20E66E4E
:102AB000D950010FE96E000EEED981EC1AF0006ECC
:102AC000060EE15C02E2E16AE552E16E0050DF6E63
:102AD000840EDF1405E0210E0101326F336B0FDA33
:102AE000D950FA0FE96EFF0ED6D945EC1DF0E5522C
:102AF000E552E552E552190E1CC0DBFF1A0E1DC04F
:102B0000DBFF1B0E1EC0DBFF1C0E1FC0DBFF95D9B9
:102B100002DA390E36DA35EC14F0010A07E108DA88
:102B2000D950190FE96E000EC1D931D186D9F3D928
:102B30001EDA06E1E4D9210E0101326F336B52D166
:102B40007CD9226A236A246A12DA01E079D0F90E6C
:102B5000DBCFE6FF010EE552D880E754E76E0C0E9E
:102B6000E7CFDBFF006A016A026A3F0E036E086A64
:102B7000096A800E0A6E3F0E0B6E190EDBCF0CF049
:102B80001A0EDBCF0DF01B0EDBCF0EF01C0EDBCFD1
:102B90000FF00CC022F00DC023F00EC024F00FC0C7
:102BA00025F008C01DF009C01EF00AC01FF00BC0C0
:102BB00020F088EC12F0C3D988D920C0DBFF006A6E
:102BC000016A026AC00E036E00C0E6FF01C0E6FFA4
:102BD00002C0E6FFE66ED9501D0FE96E000E5BD90C
:102BE000C4EC17F0E552E552E552E552E552E7CF65
:102BF00003F0E552E7CF02F0E552E7CF01F0E552EE
:102C0000E7CF00F01CC004F01DC005F01EC006F0A8
:102C10001FC007F01CC022F01DC023F01EC024F00E
:102C20001FC025F0F4D872EC13F0190E1DC0DBFFA5
:102C30001A0E1EC0DBFF1B0E1FC0DBFF1C0E0FD0C9
:102C400077D950D9190EDBCF22F01A0EDBCF23F043
:102C50001B0EDBCF24F01C0EDBCF25F036D920C0B5
:102C6000DBFF1D0EDBCF04F01E0EDBCF05F01F0EC9
:102C7000DBCF06F0200EDBCF07F00B0E226E8D0EA1
:102C8000236EB10E246EC00E256E04C01DF005C06B
:102C90001EF006C01FF007C020F089EC12F0E7D844
:102CA000F00E226E500E236EB30E246E400E256E73
:102CB00089EC12F0110E1DC0DBFF120E1EC0DBFFEF
:102CC000130E1FC0DBFF140E20C0DBFF650E1D6E50
:102CD000200E1E6E010E1F6EBF0E206EC8D86B0E2A
:102CE000226E160E236E6F0E246E3F0E256E89EC3B
:102CF00012F00D0E1DC0DBFF0E0E1EC0DBFF0F0E0F
:102D00001FC0DBFF100E20C0DBFF1D0EDBCF1DF050
:102D10001E0EDBCF1EF01F0EDBCF1FF0200EDBCF11
:102D200020F00D0EDBCF22F00E0EDBCF23F00F0EC6
:102D3000DBCF24F0100E21D9110EDBCF22F0120EC2
:102D4000DBCF23F0130EDBCF24F0140EDBCF25F006
:102D50001FEC13F0150E1DC0DBFF160E1EC0DBFFAF
:102D6000170E1FC0DBFF180E20C0DBFF66D8BAD8D5
:102D7000150EDBCF22F0160EDBCF23F0170EDBCFC4
:102D800024F0180EFAD8DBD889EC12F063D8F90ECB
:102D9000DB500EE10C0EDB5006E042D8C1D8F1D872
:102DA00089EC12F057D80B0EDB501CE0DAD819D0A2
:102DB0000B0EDB500CE00C0EDB500EE131D8DB0EBD
:102DC000226E0F0E236E490E246E400E07D0C9D816
:102DD00041D80C0EDB5006E023D8A2D8D2D889EC1B
:102DE00012F038D81DD800C01CF001C01DF002C080
:102DF0001EF003C01FF0210EE15C02E2E16AE55221
:102E0000E16EE552E5CFDAFFE7CFD9FF120000C04F
:102E10001DF001C01EF002C01FF003C020F0120020
:102E2000010EDBCF00F0020EDBCF01F0030EDBCF93
:102E300002F0040EDBCF03F01200190EDBCF00F01E
:102E40001A0EDBCF01F01B0EDBCF02F01C0EDBCF26
:102E500003F01200010E1DC0DBFF020E1EC0DBFFDF
:102E6000030E1FC0DBFF040E20C0DBFF12001D0E8F
:102E7000DBCF22F01E0EDBCF23F01F0EDBCF24F0C2
:102E8000200E7BD81DC000F01EC001F01FC002F054
:102E900020C003F01200DA20EA6EEECFE6FFEECF9C
:102EA000E6FFEECFE6FFEFCFE6FF1200DA20EA6E94
:102EB000010EEECFDBFF020EEECFDBFF030EEECFF7
:102EC000DBFF040EEECFDBFF120072EC13F01D0EE1
:102ED0001DC0DBFF1E0E1EC0DBFF1F0E1FC0DBFF71
:102EE000200E1200190EDBCF1DF01A0EDBCF1EF0E4
:102EF0001B0EDBCF1FF01C0EDBCF20F01200010EEB
:102F0000DB68020EDB68030EDB687F0EF36E040ED7
:102F1000F3CFDBFF1200226A236A800E246E1200B8
:102F2000DB0E226E0F0E236EC90E246E3F0E1200B2
:102F3000F90EDB50E76E0C0EE7CFDBFF12001DC071
:102F400004F01EC005F01FC006F020C007F01DC031
:102F500022F01EC023F01FC024F020C025F007EF90
:102F600017F05EDFD8DFBF0E0CD872EF13F03F0E04
:102F700008D82CEC14F0010A1200DBCF25F072EF18
:082F800013F0256E07EF17F0B6
:082F8800D9CFE6FFDACFE6FF26
:102F9000E1CFD9FFE2CFDAFF240EE12402E3E168BA
:102FA000E652E16ED950FA0FE96EFF0EDA20EA6EB2
:102FB000020EEECFDBFF030EEECFDBFF040EEECFF3
:102FC000DBFF050EEECFDBFFE8D9F2D981EC1AF07A
:102FD000006E060EE15C02E2E16AE552E16E00502D
:102FE000E76E0D0EE7CFDBFFDB50800815E0A0D9C0
:102FF000226A236A246A256A00C01DF001C01EF0FF
:1030000002C01FF003C020F035EC14F0010A10E1FB
:10301000210E0101326F336B020EDB68030EDB6899
:10302000040EDB687F0EF36E050EF3CFDBFF66D177
:103030000D0EDB50050B01E061D10A0EDBCF00F075
:103040000B0EDBCF01F0830E0026FF0E012200C025
:10305000DEFF01C0DDFFD950060F65D976D9DF50FC
:10306000010B0FE0DF06010E01E2DB06D950180F5D
:103070005AD9D890EF36010EEB36020EEB36030E1E
:10308000EB36D9CFE9FFDACFEAFF020E236E246ACE
:10309000EECF1EF0EDCF1FF019EC15F01EC0EEFFC5
:1030A0001FC0EDFF140EDB6A150EDB6A160EDB6A1D
:1030B000170EDB6A1C0EDB6A1D0EDB6A1E0EDB6A56
:1030C000010EF36E1F0EF3CFDBFF010EF36E0E0E3B
:1030D000F3CFDBFF0F0EDB6A0E0EDBCF00F00F0E1F
:1030E000DBCF01F0D890015004E61A0E005C000E10
:1030F000015801E398D0180EDBCF00F0190EDBCF9A
:1031000001F01A0EDBCF02F01B0EDBCF03F0010E35
:103110001F0B07E0D8900036013602360336E8066A
:10312000F9E1180E00C0DBFF190E01C0DBFF1A0E1B
:1031300002C0DBFF1B0E03C0DBFF140EDBCF08F069
:10314000150EDBCF09F0160EDBCF0AF0170EDBCF22
:103150000BF0010E1F0B07E0D890083609360A362F
:103160000B36E806F9E1D9501C0FDDD80850EE24E3
:10317000046E0950EE20056E0A50EE20066E0B50CC
:10318000EE20076ED950180FCED80450EE5C006EBA
:103190000550EE58016E0650EE58026E0750EE587C
:1031A000036E200E00C0DBFF210E01C0DBFF220EEC
:1031B00002C0DBFF230E03C0DBFF200EDBCF1DF0C0
:1031C000210EDBCF1EF0220EDBCF1FF0230EDBCF54
:1031D00020F02034000E201809E6D880000E1D547F
:1031E000000E1E54000E1F54000E205411E2D95040
:1031F000200F99D8AAD8D8D81C0EDB50EE121D0E7D
:10320000DB50EE121E0EDB50EE121F0EDB50EE12E4
:10321000D9501C0F88D8AFD80E0EDB2A0F0E01E252
:103220005BD7DB2A59D7C9D8100E00C0DBFF110EBF
:1032300001C0DBFF180EDBCF1EF0190EDBCF1FF035
:10324000120E1EC0DBFF130E1FC0DBFFADD893D8DC
:10325000D950100F68D8EE50ED1012E0D950120F6F
:1032600062D8EE50ED1006E1A8D80050011002100F
:10327000031006E099D8EE2A000EEE22EE22EE228E
:103280000C0EDB6A91D8060EEECFDBFF070EEECFF9
:10329000DBFF080EEECFDBFF090EEECFDBFF7E0E6D
:1032A000F36E0A0EF3CFDBFF0B0EDB6AD950020F71
:1032B000E66E000EDA20E66E70D80FEC1BF0E552D9
:1032C000E552E552E552DECFE6FFDDCFE6FF70D8EE
:1032D000E5EC19F0006E060EE15C02E2E16AE552EF
:1032E000E16E0050020E1CC0DBFF030E1DC0DBFFB1
:1032F000040E1EC0DBFF050E1FC0DBFF19D800C087
:103300001CF001C01DF002C01EF003C01FF0240E0F
:10331000E15C02E2E16AE552E16EE552E5CFDAFFF7
:10332000E7CFD9FF1200E96E000EDA20EA6E120034
:10333000020EDBCF00F0030EDBCF01F0040EDBCF7B
:1033400002F0050EDBCF03F01200180EEECFDBFF0C
:10335000190EEECFDBFF1A0EEECFDBFF1B0EEECF0A
:10336000DBFF1200EECFE6FFEECFE6FFEECFE6FF8B
:10337000EFCFE6FF1200D890030EEB32020EEB32D5
:10338000010EEB32EF321200EE500016EE50011635
:10339000EE500216EE5003161200D950060FE66EDC
:1033A000000EDA20E66E1200D950140F93EF19F0D8
:1033B000D950020FB8DFB2EF19F0010E006E016AAA
:0A33C000026A036AF1DFC4EF19F09E
:0633CA0096D8E1CFD9FF07
:1033D000E2CFDAFF0C0EE12402E3E168E652E16E8F
:1033E000D950FA0FE96EFF0EDA20EA6E080EEECF22
:1033F000DBFF090EEECFDBFF0A0EEECFDBFF0B0E7D
:10340000EECFDBFF79D8D950080FE96E000EDA2035
:10341000EA6EEECFE6FFEECFE6FFEECFE6FFEFCFB0
:10342000E6FF81EC1AF0006E060EE15C02E2E16A52
:10343000E552E16E0050E76E070EE7CFDBFFDB5091
:10344000840B3AE1070EDB041AE1060EDB5006E0BE
:10345000006A016A026A800E036E04D0006A016A83
:10346000026A036A080E00C0DBFF090E01C0DBFF21
:103470000A0E02C0DBFF0B0E03C0DBFF1DD0F80EEF
:10348000DBCF00F0F90EDBCF01F0D950040FE96E6D
:10349000000EDA20EA6E0050EE260150ED22D950DF
:1034A000080FE66E000EDA20E66E26D80FEC1BF051
:1034B000E552E552E552E552080EDBCF00F0090E69
:1034C000DBCF01F00A0EDBCF02F00B0EDBCF03F0F7
:1034D00000C01CF001C01DF002C01EF003C01FF0B0
:1034E0000C0EE15C02E2E16AE552E16EE552E5CFE5
:1034F000DAFFE7CFD9FF1200D9CFE6FFDACFE6FF38
:023500001200B7
:0E350200D9CFE6FFDACFE6FFE1CFD9FFE2CF67
:10351000DAFFE652006801687F0E026E036AD95036
:10352000FA0FE96EFF0EDA20EA6EEE500016EE504A
:103530000116EE500216EE5003166AD800C0EEFFD8
:1035400001C0EEFF02C0EEFF03C0EEFFFD0EDB5038
:10355000800B02E0010E01D0000EE66E59D8060E77
:10356000E926000EEA22E552E750EF6EFC0EDBCFB3
:1035700000F0FD0EDBCF01F0D89000360136FC0ED6
:1035800000C0DBFFFD0E01C0DBFFDB50E66E40D864
:10359000040EE926000EEA22E552E750EE6EED6ACF
:1035A000FD0EDB50006E016AFF0E001818E101509D
:1035B00016E12ED8EECF00F0EECF01F0EECF02F004
:1035C000EFCF03F0005001100210031006E0210EAF
:1035D0000101326F336B800E0BD0040E09D0FD0E4B
:1035E000DB5008E115D8EE6AEE6AEE6AEE6A010E6B
:1035F000DF6E06D0020EDF6E0BD8EE52EE52EE8E6C
:10360000DF50E552E552E5CFDAFFE7CFD9FF1200F0
:0E361000F80EDBCFE9FFF90EDBCFEAFF120068
:02361E00D9CF02
:10362000E6FFDACFE6FFE1CFD9FFE2CFDAFF5BD8E2
:10363000013411E20050FE08000E01540CE276D86D
:1036400005E06CD8800EEE6EEE6847D067D8800E2D
:10365000EE6E7F0E0ED047D8D890015004E6010ED2
:10366000005C000E01580BE261D805E057D8EE6A05
:10367000800EEE6E32D052D8EE6AEE6A2ED047D867
:10368000EECF00F0EECF01F0EECF02F0EFCF03F07F
:1036900032D800C0EEFF01C0EEFF02C0EEFF03C053
:1036A000EEFF21D80050010B05E025D8020E3AD8D4
:1036B000EF8E04D020D8020E35D8EF9E14D8D890C3
:1036C0000132003218D8030E2DD800C0EFFF1AD8EF
:1036D00004E011D8030E26D8EF8EE552E5CFDAFFCD
:1036E000E7CFD9FF120013D8040E1CD8EECF00F09C
:1036F000EFCF01F01200FA0EDBCFE9FFFB0EDBCFBC
:10370000EAFF120004D8060E0DD8EF501200FC0E8E
:10371000DBCFE9FFFD0EDBCFEAFF1200ECDFEE6A44
:10372000EE6A1200E926000EEA221200220E0101C2
:08373000326F336B82EF1BF0D6
:08373800040120511F0B0108E0
:1037400001E06DD0245101E06AD0060E215D28E130
:103750002351230A21E0010A11E0030A01E020D0ED
:10376000010101050AE10101480E116F380E126FC7
:10377000090E146F156BC00E136F12D001010105F5
:103780000AE10101A10E116F380E126F4A0E146F7B
:10379000156BC00E136F04D00101800E136F00D0A3
:1037A00004012051600BE842E842E842E842E84266
:1037B000010801E034D021510B0A2BE0080A1EE079
:1037C000090A16E0080A09E00B0A05E0080A01E008
:1037D00026D026D824D025D822D001012F0E116F53
:1037E000010E126F010E146F156BC10E136F17D0FF
:1037F0000101800E136F23C42FF111D00101300E8F
:10380000116F010E126F010E146F156B810E136F85
:1038100006D00101800E136F22C430F100D01200D7
:043820001200120080
:0C382400120100020000000879000F5D96
:103830000300010200010902290001010080320990
:103840000400000203000000092111010001224AC6
:10385000000705810340000A0705010340000A0430
:10386000030904120353007400610072006C0069C4
:10387000006E006F002C0353007400610072006C36
:103880000069006E006F002000470061006D006558
:10389000007000610064002000760031002E0035C9
:1038A0000005010905A1010901A10209300931152D
:1038B0000026FF00750895028102050919012908F3
:1038C000150025017501950881027508952126FFCF
:1038D000000600FF09018102C0A10275089521269A
:1038E000FF000600FF09029102C0C036385F38634E
:0338F000387538F0
:0C38F400060EF66E000EF76E000EF86E69
:1039000001010900F5502A6F0900F5502B6F03E102
:103910002A6701D03DD00900F550256F0900F55008
:10392000266F0900F550276F09000900F550E96E70
:103930000900F550EA6E090009000900F550286FEA
:103940000900F550296F09000900F6CF2CF1F7CFD7
:103950002DF1F8CF2EF125C1F6FF26C1F7FF27C1C3
:10396000F8FF0101285302E1295307E00900F5504F
:10397000EE6E2807F8E22907F9D72CC1F6FF2DC112
:10398000F7FF2EC1F8FF01012A07000E2B5BBFD7FE
:02399000120023
:0E399200D9CFE6FFDACFE6FFE1CFD9FFE2CFD3
:1039A000DAFFAC6AAB6AFD0EDBB0AC88DBA202D0FA
:1039B000AC8CAB8CDBB4AC8EDBA602D0AB8801D078
:1039C000AB8ADBB8AC849E98DBBAAB86DBAC02D0AA
:1039D0009D8A01D09D9A9E9ADBAE02D09D8801D02F
:1039E0009D98FB0EDB50AF6EFB0EFC0EDBCF01F0A3
:1039F00001C000F0016A0050B06EAC8AAB8E949C9E
:103A0000948EAC50100B04E0AC50800B01E1948C10
:0C3A1000E552E5CFDAFFE7CFD9FF120046
:043A1C00D9CFE6FF19
:103A2000DACFE6FFE1CFD9FFE2CFDAFFC26AC06AA0
:103A3000FC0EDB407F0B3C0BC26EFB0EDBCFE6FFC8
:103A4000FC0EDB38F00B300BE552E710C16EFD0EBB
:103A5000DB50040DF350380B016EFD0EDB380F0BFD
:103A6000070B006EFD0EDB50800B00100110C06EC6
:103A7000FC0EDBAE03D09E9C9D8CF28CC280E55286
:0A3A8000E5CFDAFFE7CFD9FF12000F
:063A8A00D9CFE6FFDACF00
:103A9000E6FFE1CFD9FFE2CFDAFFE652E652D95096
:103AA000FD0F006EFF0EDA2000C0DEFFDD6EDECF00
:103AB000E9FFDDCFEAFFEF9EFA0EDBCF00F0FB0E51
:103AC000DBCF01F0FC0EDBCF02F0FD0EDBCF03F00D
:103AD00000C01CF001C01DF002C01EF003C01FF0AA
:103AE000E552E552E552E5CFDAFFE7CFD9FF120004
:103AF000D9CFE6FFDACFE6FFE1CFD9FFE2CFDAFF99
:103B0000E66AD950FA0FE96EFF0EDA20EA6EEECFC0
:103B1000E6FFEECFE6FFEECFE6FFEFCFE6FF3FECAE
:103B200015F0006E050EE15C02E2E16AE552E16E1D
:0E3B30000050E552E5CFDAFFE7CFD9FF1200D3
:023B3E00D9CFDD
:103B4000E6FFDACFE6FFE1CFD9FFE2CFDAFFFF0EE3
:103B5000E76EFC0EDBCF00F0E75000160050A96EB8
:103B6000FB0EDB50A86EA69EA69CA684F29E550E68
:103B7000A76EAA0EA76EA682F28EA694E552E5CF96
:083B8000DAFFE7CFD9FF1200C4
:083B8800D9CFE6FFDACFE6FF1A
:103B9000E1CFD9FFE2CFDAFFE652E652D650DF6E30
:103BA000010ED7CFDBFFDECF00F0DDCF01F000C08C
:103BB000F3FF01C0F4FFE552E552E552E5CFDAFF2D
:063BC000E7CFD9FF12005F
:0A3BC600D9CFE6FFDACFE6FFE1CF2A
:103BD000D9FFE2CFDAFFFD0EDB507F0BD56ED76A3F
:103BE000D66AF294FD0EDBAE02D0F28A01D0F29AD0
:0E3BF000D58EE552E5CFDAFFE7CFD9FF120000
:023BFE00D9CF1D
:103C0000E6FFDACFE6FFE1CFD9FFE2CFDAFFFF0E22
:103C1000E76EFC0EDBCF00F0E75000160050A96EF7
:103C2000A69CA69EA680A850E552E5CFDAFFE7CF76
:043C3000D9FF1200A6
:0C3C3400FE0EE3CFE9FFFF0EE3CFEAFF36
:103C4000E9CFF3FFEACFF4FFFB0EE35003E1FC0EF4
:103C5000E35009E0FB0EE30602E2FC0EE306FD0E74
:083C6000E350EE6EF1D71200F3
:083C6800D9CFE6FFDACFE6FF39
:103C7000E1CFD9FFE2CFDAFFACAC04D0AC900101C8
:103C800034B3AC80FD0EDB50AD6EE552E5CFDAFF0C
:063C9000E7CFD9FF12008E
:0A3C9600D9CFE6FFDACFE6FFE1CF59
:103CA000D9FFE2CFDAFFC30EC214006EFD0EDB4077
:103CB0007F0B3C0B0010C26EE552E5CFDAFFE7CF79
:043CC000D9FF120016
:0C3CC4001B6A1A6A100EE76ED8901E36BC
:103CD0001F361A361B3623501A5C24501B5805E336
:103CE00023501A5E24501B5A1E2AE72EF0D71200CA
:103CF000FF0EE3502A6E480E01D04C0EE76EE72E01
:103D0000FED7E76AE72EFED72A2EF7D7000012006B
:103D100013EE00F023EE00F0F86A179C7AEC1CF02A
:0C3D2000BBEC1EF090EC08F0FBD712008A
:043D2C00FF0EE35053
:103D3000E84E1200000000D000D000D0E82EFAD7E4
:023D400012006F
:0E3D4200C450036E026AC3500210F36E03C039
:043D5000F4FF12006A
:0C3D540000EE00F00F0EEE6AEA62FDD7F0
:023D600012004F
:0A3D6200C250020B01E0010E120036
:043D6C00A6B2FED726
:023D700012003F
:043D7200C2821200F7
:023D7600120039
:063D780000000000000045
:020000040030CA
:0100000024DB
:010001000EF0
:010002003FBE
:010003001EDE
:0100050001F9
:010006008178
:010008000FE8
:01000900C036
:01000A000FE6
:01000B00E014
:01000C000FE4
:01000D0040B2
:00000001FF
